:100000000C9414020C9467020C9467020C9467021F
:100010000C9467020C9467020C9467020C946702BC
:100020000C9467020C9467020C9475280C94670278
:100030000C944C280C9467020C9467020C94670291
:100040000C9467020C9467020C9467020C9467028C
:100050000C9467020C94D02B0C9467020C946702EA
:100060000C9467020C9467020C9467020C9467026C
:100070000C9467020C9467020C9467020C9467025C
:100080000C9467020C9467020C9467020C9467024C
:100090000C9467020C9467020C9467020C9467023C
:1000A0000C9467020C9467020C9467020631FF09F6
:1000B00074A1010975150026FF00952075088102BD
:1000C0000976150026FF00952075089102C00501EC
:1000D0000902A1010901A1008501050919012908E9
:1000E00015002501950875018102050109300931C6
:1000F0001581257F95027508810609381581257FB0
:10010000950175088106050C0A38021581257F9531
:100110000175088106C0C005010980A1018502168C
:1001200001002637001A81002AB700751095018159
:1001300000C0050C0901A1018503160100269C02DF
:100140001A01002A9C02751095018100C005010961
:1001500006A101050719E029E71500250195087595
:10016000018102950175088101050819012905958C
:100170000575019102950175039101050719002983
:10018000FF150026FF00950675088100C073706595
:1001900065643A2025730A007573625F7374617435
:1001A000653A20253032580A00686F73742E546106
:1001B000736B3A2025640A00526F6C6C6F7665721F
:1001C000206572726F723A2069676E6F7265640D96
:1001D0000A000D0A00202530325800696E707574CF
:1001E0002025643A000A4C6F6F702073746172743A
:1001F0002E0A000A55534220636F6E666967757256
:1002000065642E0A000A544D4B3A316631666535F5
:100210002F4C5546413A6436613764662F55485332
:10022000323A3864376563660A00090254000301F4
:1002300000A032090400000103010100092111019D
:1002400000012240000705810308000A090401009B
:100250000103010200092111010001227F000705AD
:1002600082030800010904020001030000000921C3
:100270001101000122220007058303200001120161
:10028000100100000008EDFE5B00150801020001EE
:100290003C03550053004200200074006F00200012
:1002A00055005300420020006B0065007900620099
:1002B0006F00610072006400200063006F006E0038
:1002C000760065007200740065007200000008038B
:1002D00054004D004B00000004030904808080801E
:1002E0000405060708090A0B0C0D0E0F1011121356
:1002F0001415161718191A1B1C1D1E1F2021222346
:100300002425262728292A2B2C2D2E2F3031323335
:100310003435363738393A3B3C3D3E3F4041424325
:100320004445464748494A4B4C4D4E4F5051525315
:100330005455565758595A5B5C5D5E5F6061626305
:100340006465736768696A6B6C6D6E6F70717273E8
:100350008080808080808080808080030201808017
:100360008066807500747677808080807677808064
:10037000808080808080808080808080808080807D
:10038000808080808080808080808080808080806D
:10039000808080808080808080808080808080805D
:1003A000808080808080808080808080808080804D
:1003B00080808080808080808080808078797A7B57
:1003C0007C7D7E7F80808080808080808080808037
:1003D000808080808080808080808080290A0025C5
:1003E00075002F002575005D28002564002000257C
:1003F0006400200025640020002564007C00253076
:100400003258006D6F7573656B6579205B62746E31
:100410007C782079207620685D287265702F616372
:100420006C293A205B005A2711241FBECFEFDAE077
:10043000DEBFCDBF04B603FE28C08091CF059091EA
:10044000D005A091D105B091D2058730904BA7403F
:10045000B04BD9F41092CF051092D0051092D1056F
:100460001092D20514BE0FB6F894A8958091600042
:10047000886180936000109260000FBE10920108A6
:1004800010920008E0E0F8E3099511E0A0E0B1E087
:10049000EAE0FBE502C005900D92A439B107D9F757
:1004A00025E0A4E9B1E001C01D92AF3CB207E1F73D
:1004B00012E0C4E1D2E004C02197FE010E94692D40
:1004C000C331D107C9F70E944F290C94832D0C9496
:1004D0000000FF93EF93E0919401F0919501309724
:1004E00009F00995EF91FF910895FC018591803005
:1004F00011F0EFDFFBCF0895FF27E0E230E247FF86
:100500000CC0419597FF09C0EDE26095709580950C
:100510009095611D711D811D911D27FF02C02195C0
:1005200030E350E2AA27660F771F881F991FAA1F82
:10053000A41710F0A41B63955A95A9F7AA3008F0E8
:10054000A95FA05DAF93F3956115710581059105D4
:1005500041F7ED3211F4EF93F395F21718F43F934E
:10056000F395FBCF8F91B5DFFA95E1F70895E99107
:10057000F9918591803021F0853219F0AADFF9CF09
:10058000089520E0E89455915532C1F3503311F4A9
:10059000689455915A3348F4505390F3220F022E29
:1005A000220F220F200D250FF4CF0EF421958991F3
:1005B0009991533619F3533729F1533559F1BC0149
:1005C00088279927E8945C3621F489919991689459
:1005D0005591543639F446EF7EF077FF0DC08FEF1A
:1005E0009FEF0AC055374AE039F0583540E121F015
:1005F000523642E009F00895FF93EF937DDFEF91CB
:10060000FF91B7CFFF93EF93FC0181918030B9F355
:1006100060DFFBCFFF93EF9368DFF1CFDF93CF93E2
:10062000CDB7DEB72596A3DFCF91DF910895FC010A
:1006300088E595E0958384838BE391E091838083C3
:1006400089E591E093838283148A158A168A178A32
:10065000108E128E81E0838B128A108A178288E0B6
:1006600080878CE381871286138684E084871586D1
:100670001686AEEAB5E090E080E02D913D91232B07
:1006800041F4880F991FDC01A255BA4FED93FC93FA
:10069000089501968031910581F7089580913C0479
:1006A00080FD16C081FD16C082FD16C080913D04FC
:1006B0008823A1F0883280F428E0829FC0011124B1
:1006C00068E270E00E94552D862F672B39F008955F
:1006D00082E0089584E0089588E0089581E0089517
:1006E00080913C0480FD14C081FD14C082FD16C0C1
:1006F00080913D04882381F0843180F422E3829F3D
:10070000C001112464E170E00E94552D862F0895E8
:100710008CE0089589E1089585E0089582E30895C5
:1007200020E1729FF0011124E60FF11DE452FD4F0C
:100730006491E62FE295E77028E0829FC0011124C2
:100740008E0F911D24E0880F991F2A95E1F7E62F5F
:10075000EF70E80FF92FF11DEE0FFF1FE050F84981
:10076000859194910895E6E9F2E09281891301C0A0
:100770001282319692E0EC39F907B9F70895A8E9A9
:10078000B2E0EFEF90E02D91821751F0EF3F19F4B6
:10079000211101C0E92F9F5F9630A9F7EF3F09F4BF
:1007A00008950E2E000CFF0BEA56FD4F828308952C
:1007B0008091360490913504892B80939602909114
:1007C0003404992381F0892B80939602E7E9F2E0C3
:1007D00080E0919191118F5F92E0EE39F907C9F7AE
:1007E000811110923404E0913F04F091400430975D
:1007F00031F00280F381E02D86E992E009940895BA
:100800004F925F926F927F929F92AF92BF92CF92E0
:10081000DF92EF92FF920F931F93CF93DF9300D05D
:1008200000D01F92CDB7DEB76B837C838D837A01B6
:100830008C819D81892B49F08FEFF81204C081E0F3
:100840009FEF491719F080E001C081E080FD6AC088
:100850000F2D10E0CE2CD12C8B81882309F456C0AB
:100860004090300350903103609032037090330316
:1008700080912C0390912D03A0912E03B0912F0312
:10088000482A592A6A2A7B2A2FE1A22EB12C9A2CB7
:10089000D301C2010A2C04C0B695A79597958795F8
:1008A0000A94D2F780FD2BC081E0A81AB10878F72E
:1008B000912CF80194E0EE0FFF1F9A95E1F7EC5CA4
:1008C000FC4FEC0DFD1D9082E982FA8269817A81EC
:1008D000892D0F900F900F900F900F90DF91CF9177
:1008E0001F910F91FF90EF90DF90CF90BF90AF904E
:1008F0009F907F906F905F904F900C949003B70102
:100900008A2D0E949003019779F2D3CFF80184E0F9
:10091000EE0FFF1F8A95E1F7EC5CFC4FEC0DFD1D1F
:100920009080D2CF90E080E00F900F900F900F90CA
:100930000F90DF91CF911F910F91FF90EF90DF907B
:10094000CF90BF90AF909F907F906F905F904F90AF
:10095000089541E050E060E070E004C0440F551F8E
:10096000661F771F8A95D2F74095509560957095D0
:100970008091300390913103A0913203B091330301
:1009800084239523A623B7238093300390933103C8
:10099000A0933203B0933303089541E050E060E048
:1009A00070E004C0440F551F661F771F8A95D2F769
:1009B0008091300390913103A0913203B0913303C1
:1009C000842B952BA62BB72B809330039093310368
:1009D000A0933203B0933303089580912B03909139
:1009E000FA02981301C008958F5F8770FACF1F93A2
:1009F000CF93DF9300D000D01F92CDB7DEB7942FF6
:100A00004983252F5A836B837C838D834C815D8141
:100A100081E0452B31F02F3F19F481E09F3F09F031
:100A200080E0182F117080FD2CC049815A816B81A4
:100A30007C818D810E940004292F22952F702C30FB
:100A400078F42A30A8F422502230C8F0812F0F9079
:100A50000F900F900F900F90DF91CF911F910895FD
:100A60002C3011F02F3091F793FB112710F9EECFB6
:100A7000803C28F0803E50F3815F833038F311E0F2
:100A8000E5CF10E0E3CF882341F0809590913604C4
:100A90008923809336040C94D8030895882339F071
:100AA00090913604892B809336040C94D8030895D2
:100AB0002091F2023091F3022817390771F09093D8
:100AC000F3028093F202E0913F04F09140043097EA
:100AD00021F00084F185E02D099408952091F00221
:100AE0003091F1022817390771F09093F102809349
:100AF000F002E0913F04F0914004309721F006802D
:100B0000F781E02D09940895E0913F04F0914004AD
:100B1000309721F00190F081E02D099480E0089554
:100B2000E8EDF0E080818E7F80831092E2001092E9
:100B3000DA001092E100A0EEB0E08C9181608C931D
:100B400080818F77808319BCA7EDB0E08C918E7F78
:100B50008C9380818F7E80831092D8020895FC014F
:100B60008091ED029091EE0286179707A0F0611533
:100B7000710529F49091E8009E779093E80090E049
:100B80006115710551F4911108C08091E80082FF50
:100B900035C080E00895BC01F2CF8091EF02882338
:100BA000C9F18530C9F18091E80083FD31C08091A1
:100BB000E80082FDEACF8091E80080FFE1CF20913C
:100BC000F3008091F200322F282F6115710519F082
:100BD0002830310558F091E02830310509F090E0D7
:100BE0002091E8002E772093E800CACF819180936E
:100BF000F100615071092F5F3F4FE7CF8091EF0205
:100C0000882341F0853041F08091E80083FFBDCF1B
:100C100081E0089582E0089583E008952091E40042
:100C20003091E50085E69091EC0090FF06C0909130
:100C3000E80090FF06C080E008959091E80092FDE2
:100C4000FACF9091EF02992391F0953091F0909125
:100C5000EB0095FD10C04091E4005091E500241791
:100C6000350709F381509A01F1F684E0089582E096
:100C7000089583E0089581E008958091E70287FF59
:100C800013C08091E80082FF06C08091E8008B7756
:100C90008093E80004C08091EF028111F2CF0895A3
:100CA0008091EF028823D9F38091E80080FFF8CF8C
:100CB0008091E8008E77ECCF982F9093E900242F55
:100CC000762F50E0891731F07091EC002091ED0003
:100CD0005091F00021FD07C09F5F973071F780931E
:100CE000E90081E008953091EB003E7F3093EB0006
:100CF0003091ED003D7F3093ED003091EB0031609D
:100D00003093EB007093EC002093ED005093F000D3
:100D10002091EE0027FDE0CF80E00895CF92DF9292
:100D2000EF92FF920F931F93CF93DF93C8EDD0E024
:100D300088818F7E8883E7EDF0E080818160808309
:100D400084E082BF81E08093D80288818E7F88838F
:100D500002EE10E0F80110821092DA0081EEC82E47
:100D6000D12CF601108288818F77888388818068F2
:100D7000888388818F7D888319BC1092EF0210923E
:100D8000E6021092E5021092E40290EEE92EF12CB8
:100D9000F70180818B7F808388818160888342E036
:100DA00060E080E00E945C06F60180818E7F808397
:100DB000F801808181608083808188608083F70171
:100DC00080818E7F8083888180618883DF91CF914D
:100DD0001F910F91FF90EF90DF90CF900895809139
:100DE000DB0208950F931F93CF93DF93FC018B01D8
:100DF000EA0180819181892B31F19281992349F116
:100E000028813981232BF9F0D8012D913C91D9010A
:100E10004C918381682F691B770B80819181860FAC
:100E2000971FDC014C938281815082838881998154
:100E3000019799838883D8018D919C911197019690
:100E40008D939C93DACF80E0DF91CF911F910F912A
:100E500008958381828381E0F7CFCF93DF93EC0104
:100E60008A819B81DC01ED91FC910480F581E02D6C
:100E70006A8509958A85813439F4EA81FB81EA58CB
:100E8000FF4F80818B7F80831A861B861C861D8680
:100E90001E861F86188A80E0DF91CF91089581E039
:100EA000693009F080E00895FC0182850895DF92A1
:100EB000EF92FF920F931F93CF93DF93EC0185E0A6
:100EC000E62EF12CFE01869FE00DF11D1124908588
:100ED00096FF24C0192F177001E085E0D82E8FEF00
:100EE000800F8F3008F001E0602F70E0062FD69E53
:100EF000F001D79EF00D1124EC0FFD1F8085869523
:100F0000869586958770181701F16F5F7F4F603166
:100F100068F38D81811302C011501D8385E08E9D81
:100F2000F0018F9DF00D1124EC0FFD1F108681E064
:100F3000818712862296D783C683DF91CF911F9136
:100F40000F91FF90EF90DF900895CE010E94570718
:100F5000C6CFFC0121E0613499F49C01255B3F4F31
:100F600061E0AC014E5F5F4F158666871786548738
:100F7000438735962E173F07B9F7FC011582089570
:100F80003585631729F02F5F35962031C9F708950D
:100F9000622F0C945707CF93DF93FC0167FD12C0BB
:100FA000283080F4442319F08581873059F0EF010F
:100FB000A1E0B0E08D85882349F111962596A031F6
:100FC000B105C1F780E018C085E08A9FE0018B9FE2
:100FD000D00D1124CE0FDF1F442389F081E48887D0
:100FE00085818F5F858325E02A9FC0012B9F900D0F
:100FF0001124E80FF91F8085DF91CF91089581E0DA
:101000008887F1CF2770687B622B0FC06623E1F2DF
:101010006770660F660F660F4423A1F360648581D5
:101020008F5F85838770687F682B25E02A9FC001CA
:101030002B9F900D1124E80FF91F6087862FDCCFBE
:10104000FC0121E0611102C0069608953585631701
:1010500039F02F5F35962031C9F790E080E0089590
:10106000069635E0239F800D911D112408950F935E
:101070001F93CF93DF932115310599F0E901042FD8
:10108000162F0E942008FC0186ED309729F012836C
:10109000D183C083038380E0DF91CF911F910F91B3
:1010A000089588EDF9CF81E008952FB7F894609105
:1010B0003704709138048091390490913A042FBF1D
:1010C0000895CF93C091B402C1110BC00E9455087E
:1010D000643C79408105910520F081E08093B40261
:1010E000C1E08C2FCF9108952FB7F89480913704E9
:1010F00090913804A0913904B0913A042FBF08951B
:10110000EF92FF920F931F93CF93DF93D82F0FB6D9
:1011100007FE46C08091EF02843079F08091030190
:1011200090E001962091050130E0822393232091E5
:1011300004012817190609F0D0C00E946108811126
:101140000FC08091030190E001962091050130E0ED
:1011500082239323209104012817190609F0BDC0AA
:101160000E9474088C01C091E900CF708091EC005E
:1011700080FD38C080E0C82B83E08093E90085E0E3
:10118000E82E8091EB0085FD08C08091EB0080FF88
:1011900004C08091EE0087FD45C0CF70C093E90088
:1011A000E09103018E2F90E001962091050130E03F
:1011B00082239323209104012817190609F460C0A3
:1011C0008091010190910201E80FF92FF11DD08368
:1011D000809103018F5F9091050189238093030122
:1011E00081E074C080E8C7CFE0910101F091020175
:1011F000E80FF11D90818F5F20910501822380937C
:1012000004019093F1008091E80085FD0BC080916E
:10121000E80080FF07C08091E8008E778093E800A7
:10122000E09200018091040190910301981751F11F
:101230009091E80095FDD8CF80E02BC01092F1008E
:1012400034C08091030190E001962091050130E0C7
:1012500082239323209104012817190609F09DCFBA
:10126000F0900001FF2009F498CF0E9474088017C5
:10127000910709F486CFFA94F09200018C0181CF96
:1012800080E024C08091E80085FFD6CFD093F100A4
:1012900081E02091F3009091F200322F292F232B2F
:1012A00079F09091E80090FF0BC09091E80095FDD7
:1012B000C5CF9091E8009E779093E800E0920001FE
:1012C000882309F4BECFCF70C093E900DF91CF919E
:1012D0001F910F91FF90EF900895E091030170CF5F
:1012E0000E94800880E008958F929F92AF92BF92F3
:1012F000CF92DF92EF92FF920E94312C4B015C0162
:1013000020E030E04AE755E40E94C02C6B017C01EC
:1013100020E030E040E85FE30E94F62B87FD30C01C
:1013200020E03FEF4FE757E4C701B6010E94BB2C16
:101330001816F4F420E030E040E251E4C501B401B5
:101340000E94C02C0E94022C20E931E06115710539
:1013500049F4FF90EF90DF90CF90BF90AF909F90B7
:101360008F900895C9010197F1F761507109EECF8F
:10137000C701B6010E94022CCB010197F1F7E9CF1A
:1013800061E070E0F9CFEF92FF920F931F93CF933C
:10139000DF938A01EB017B01E40EF51ECE15DF051C
:1013A00021F089910E948008F9CFC801DF91CF9187
:1013B0001F910F91FF90EF900895862F0E94800853
:1013C00081E090E00895089581E090E008958FEF26
:1013D0009FEF089590E080E008953F924F925F92D2
:1013E0006F927F928F929F92AF92BF92CF92DF9235
:1013F000EF92FF920F931F93CF93DF9300D000D013
:10140000CDB7DEB76C017A8369835C834B8384E05C
:10141000482E360182E1680E711C93E0392E560188
:10142000A7E0AA0EB11C12E0552453944601B0E186
:101430008B0E911C29813A812115310509F4CDC00B
:10144000F60180A18230F1F0A8F5882309F457C095
:10145000813091F7AE014F5F5F4FBE016D5F7F4FEF
:10146000C5010E94F206882309F4B7C0D60115967B
:10147000ED91FC911697808191968C939197818143
:1014800092968C93F6017682658230A2D60192966E
:101490008C919297843011F493961C92F60181A15D
:1014A0008250848325813681308727838287818794
:1014B00040A205C0833051F3843009F0BDCFD6017E
:1014C00092968C919297843019F1853009F44BC033
:1014D000823009F075C0AE014F5F5F4FBE016D5F96
:1014E0007F4FC5010E94F206882309F476C0F601F9
:1014F000858984A3F6019682858210A29BCF1483EE
:1015000085819681908787831287118750A2A2CF09
:10151000AE014F5F5F4FBE016D5F7F4FC5010E94FF
:10152000F206882309F459C0D60155968C91559737
:10153000833001F756968C9156978130D9F698965C
:101540009C91989757968C91992351F0882391F20A
:10155000F60153A2928996A3938997A385A3CACF34
:10156000813041F6F5CFAE014F5F5F4FBE016D5F39
:101570007F4FC5010E94F206882379F1D601939628
:101580008C919397882309F4B5CF12968D919C91F5
:10159000009709F4AFCFDC01ED91FC910190F0814F
:1015A000E02D7401D60195960C91959797962C9104
:1015B000979796964C91969794966C9109959ACF99
:1015C000F60185858823F9F0813041F1D6011E9618
:1015D0008D919C91892B09F48DCF0F900F900F90D6
:1015E0000F90DF91CF911F910F91FF90EF90DF90BF
:1015F000CF90BF90AF909F908F907F906F905F90B3
:101600004F903F90089591968C9191978250990BAD
:101610001F969C938E931E971D965C9229813A810A
:101620008B819C81782F692FF6014685578541155E
:10163000510581F001962115310539F041505109CC
:101640005787468721503109EDCF1A8219827B8353
:101650006C83BCCF3A8329839C838B831586B6CF5A
:101660000895EF92FF92CF93DF93FC01E701838906
:10167000823051F1608B418B9B819370933021F5C7
:101680009A8197FF21C09E81218D291708F4918F9F
:10169000282F30E0D901AA0FBB1FA20FB31FAE0F36
:1016A000BF1F9A819F7017969C9317979C811896DD
:1016B0009C93189794E019969C932E0F3F1FD90185
:1016C0001E964C938F5F838BDF91CF91FF90EF90AD
:1016D0000895EF92FF920F9302970E94310B0F91A2
:1016E000FF90EF90089570E0660F771F860F971FA9
:1016F000FC0185859685089581E0613009F080E0E0
:10170000089581E0633009F080E00895FC0186814E
:101710000895CF93DF93EC018C819D81DC01ED91E5
:10172000FC910480F581E02D6E810995188A198A53
:1017300081E08B8B1E821C8A1D8A1E8A1F8A188E4E
:1017400080E0DF91CF9108952E9808952E9A089504
:101750000F931F93CF93DF93D82FC62F8A010E9438
:10176000A40BD260DEBDF8018C2F882339F00DB4B4
:1017700007FEFDCF91919EBD8150F7CFC00FD12FB5
:10178000D11D0DB407FEFDCF0E94A60BCE01DF9147
:10179000CF911F910F910895CF93DF93C82FD62F2C
:1017A0000E94A40BC260CEBD0DB407FEFDCFDEBD0E
:1017B0000DB407FEFDCFDF91CF910C94A60B9F9245
:1017C000AF92BF92CF92DF92EF92FF920F931F934F
:1017D000CF93DF936C01C42FD22F99249394E62EDC
:1017E000F12CEE0CFF1CE80EF91E86E5E80EF11C4C
:1017F000A42EB12CABE2AA0EB11CAA0CBB1CAC0CE3
:10180000BD1CF70180819181DC01ED91FC9102808A
:10181000F381E02D202F4D2F6C2F0995182F803E3E
:10182000C9F5C1112BC061E088EE0E94CC0B66E6C1
:1018300070E080E090E00E947409F701808191815E
:10184000DC01ED91FC910190F081E02D202F4D2FD6
:101850006C2F0995182F8D30D1F58FEF890D8330BE
:10186000F8F0C11137C061E088EE0E94CC0B66E64B
:1018700070E080E090E00E9474091CC0F501808156
:101880009181DC01ED91FC910284F385E02D6D2FB7
:101890000995D3CF8D3061F48FEF890D833050F4EB
:1018A00064E670E080E090E00E9474099394A9CF10
:1018B000882319F2812FDF91CF911F910F91FF9013
:1018C000EF90DF90CF90BF90AF909F9008958823C6
:1018D00089F3C7CF8C2F90E08B96880F991F8C0DC2
:1018E0009D1DFC0180819181DC01ED91FC910284C0
:1018F000F385E02D6D2F0995DDCFCF93C82F0E9482
:10190000A40BCEBD0DB407FEFDCF1EBC0DB407FE6B
:10191000FDCF0E94A60B8EB5CF9108958F929F9216
:10192000AF92BF92CF92DF92EF92FF920F931F93ED
:10193000CF93DF93882E962E5A010E9455086B0193
:101940007C0128E8C20E23E1D21EE11CF11CC0E09C
:1019500010E000E0D0E098280E9455086C197D093D
:101960008E099F0997FF1EC0692D80EF0E94CC0B46
:101970000E9455086C197D098E099F0997FF09C0BF
:1019800088EC0E947D0C87FFF3CF60E888EC0E9412
:10199000CC0B88EF0E947D0CC82FCF70C43081F033
:1019A000CE30B9F08C2FDF91CF911F910F91FF9026
:1019B000EF90DF90CF90BF90AF909F908F90089561
:1019C0000F5F1F4FA114B10439F20A151B0521F650
:1019D000E9CFDF5FD33009F0BFCFE4CFAF92BF9242
:1019E000CF92DF92EF92FF920F931F93CF93DF93EB
:1019F000EC01B62EA42E69010E9420087C0186ED20
:101A0000E114F10409F447C0D701ED91FC9111975D
:101A100087ED309709F43FC013969C9180E09817AA
:101A200031F02081A21629F033968F5FF8CFF0E0D5
:101A3000E0E0D601ED93FC938BED309761F12281CC
:101A400026952695203108F02FE081E090E0A0E077
:101A5000B0E004C0880F991FAA1FBB1F2A95D2F7B8
:101A60000197F801918380836B2D80EE0E94CC0B4F
:101A700088ED0E947D0CD70114969C91682F697F98
:101A8000992329F0CA58DF4F68816260682B88ED7E
:101A90000E94CC0B80E0DF91CF911F910F91FF90BE
:101AA000EF90DF90CF90BF90AF90089588EC0E94A8
:101AB0007D0C85FF14C060E288EC0E94CC0B88EF9F
:101AC0000E947D0C807C909112018917E1F1809336
:101AD0001201803409F150F4882379F1089580913E
:101AE0004804811130C064E088EEE7CF803819F0F7
:101AF000803C09F1089588ED0E947D0C9091480486
:101B000081FD11C09230F9F061EC88ED0E94CC0BA0
:101B100082E080934804089588ED0E947D0C9091A6
:101B2000480481FDEFCF933071F063EC88ED0E94A3
:101B3000CC0B83E0EECF81E0ECCF61EC88ED0E942E
:101B4000CC0B109248040895FC01808D089570E03C
:101B5000660F771F860F971FFC015687458781E028
:101B60000895482F80E1489F90011124205E31099B
:101B70002830310508F59091AB029923E9F0892FBF
:101B800090E0EDEAF2E061E070E02191243078F03D
:101B9000322F32953F7034130AC02F70DB0102C020
:101BA000AA0FBB1F2A95E2F79D018A2B932BB2E067
:101BB000E33BFB0751F7089590E080E0E2CFCF933D
:101BC000DF93CDB7DEB728970FB6F894DEBF0FBE10
:101BD000CDBFE22F29833A834B835C836D837E8361
:101BE0008F8398872091AB022E2B2093AB02FE01AE
:101BF0003396AE01475F5F4F2191243060F0ADEA2C
:101C0000B2E090E080E03D91311111C085559D4FCB
:101C1000DC0112962C93E417F50771F728960FB69E
:101C2000F894DEBF0FBECDBFDF91CF91089501962E
:101C30008630910541F7EFCF80E00895089580E068
:101C400008952F923F924F925F926F927F928F9260
:101C50009F92AF92BF92CF92DF92EF92FF920F933B
:101C60001F93CF93DF937B014A016901F901A080A3
:101C7000B180FB012180F90111821082FB01828178
:101C800060E181FD60E288EE0E94CC0B3A2CA40159
:101C9000F701608180E00E948E0C582EF6E08F17CD
:101CA000B1F381114EC088EC0E947D0C82FF5DC0B3
:101CB00080E30E947D0C482E8A151B0411F008F069
:101CC000432CF601808191813501681A790A77FEEB
:101CD00002C0712C612CC42DD0E0C615D7050CF4C0
:101CE0003E01562C0E94A40BF8E0FEBD0DB407FE89
:101CF000FDCFF801552041F01EBC5A940DB407FEEB
:101D0000FDCF8EB58193F6CF060D171D0E94A60B51
:101D100064E088EC0E94CC0BF60180819181C80FB1
:101D2000D91FD183C083421420F0CA15DB0508F403
:101D3000AECF88EF0E947D0CF701928184FB91F970
:101D40009283852DDF91CF911F910F91FF90EF909E
:101D5000DF90CF90BF90AF909F908F907F906F90CB
:101D60005F904F903F902F90089580EF582EE9CFCD
:101D7000AF92BF92CF92DF92EF92FF920F931F9399
:101D8000CF93DF9300D000D0CDB7DEB77C016901DF
:101D900058011C821B821A8219828E010F5F1F4F0D
:101DA0009E012D5F3F4F0E94EE0C811109C04981B9
:101DB0005A816B817C8185019601C7010E94210EA9
:101DC0000F900F900F900F90DF91CF911F910F9177
:101DD000FF90EF90DF90CF90BF90AF9008952F923B
:101DE0003F924F925F926F927F928F929F92AF92AB
:101DF000BF92CF92DF92EF92FF920F931F93CF93F8
:101E0000DF93CDB7DEB765970FB6F894DEBF0FBE90
:101E1000CDBF3C01342E222E402EED8AEAA4FBA435
:101E2000188A1F861E861D868E01035F1F4F9E0126
:101E3000215F3F4F40E00E94EE0C582E81111AC1E5
:101E400039822A824B822D892C83DE82CD82B8860C
:101E5000AF82AE014F5F5F4F68E080E20E94A80B47
:101E60004D855E8560E080E10E948E0C811120C16D
:101E7000E114F10409F449C00F851889D8011296BC
:101E80008C91129737FE47C0826012968C93650141
:101E9000C114D10409F411C19C2D8D2D8C149D0405
:101EA00010F4982D892D9B878C874D855E856F85D5
:101EB000788987019E01255F3F4FC3010E94210E53
:101EC000582EB6E08B1721F38111D4C0ECA5FDA5E7
:101ED0003097A1F06B857C850190F081E02D019019
:101EE000F081E02DC5018C199D099A8789879E0193
:101EF000275F3F4FA7018CA59DA509958B859C85E4
:101F0000C81AD90A8815990518F64D855E8537FED9
:101F1000CBC080EACAC0816012968C93129711964A
:101F20006C908FEF860D803408F0C4C02D843E8401
:101F30000E9455089B01AC0128573C4E4F4F5F4F04
:101F4000298B3A8B4B8B5C8BD80112968C9160E875
:101F500080FF60E488EE0E94CC0B512C712C811420
:101F6000910409F476C063018614970408F46401AF
:101F7000CD8AA7016C2D80E10E94A80B6C2D88E30F
:101F80000E94CC0BF8016081606280EF0E94CC0B54
:101F900088EC0E947D0C87FFFBCF60E888EC0E94F4
:101FA000CC0B88EF0E947D0C8F70582E412CB12CE9
:101FB000A12C552019F10E94550829893A894B898D
:101FC0005C89621B730B840B950B97FF17C036E07F
:101FD0005316E9F04EE05416B1F054E0551209C022
:101FE0008FEFA81AB80A2114310489F02A143B048F
:101FF00071F460E088E30E94CC0B2DC08C189D0822
:10200000EC0CFD1CACCF439493E0491691F360E0D7
:1020100088E30E94CC0BD7016C9180E10E94CC0B2D
:102020006D8988E30E94CC0BF8016081606280EFCB
:102030000E94CC0B88EC0E947D0C87FFFBCF60E8F0
:1020400088EC0E94CC0B88EF0E947D0C8F70582E7C
:10205000B0CF5110CECF88EF0E947D0CD8011296E0
:102060009C91129785FB90F912969C934D855E8505
:102070005520D1F0852D65960FB6F894DEBF0FBEC2
:10208000CDBFDF91CF911F910F91FF90EF90DF9027
:10209000CF90BF90AF909F908F907F906F905F9008
:1020A0004F903F902F90089580E860E00E948E0C42
:1020B000582EE0CF8AED582EDDCF4D855E85552018
:1020C00009F427CFD7CF8F929F92AF92BF92CF9232
:1020D000DF92EF920F93CF931F921F921F921F9246
:1020E000912C812CB12CA12CD12CC12CE12C062FB0
:1020F00025E040E060E00E94EF0EC82F6CE271E046
:1021000080E090E00E9474090F900F900F900F9064
:102110008C2FCF910F91EF90DF90CF90BF90AF9029
:102120009F908F9008958F929F92AF92BF92CF927F
:10213000DF92EF920F931F921F923F932F934A01CA
:102140005A01D12CC12CEE24E39400E026E040E8B3
:102150000E94EF0E0F900F900F900F900F91EF9045
:10216000DF90CF90BF90AF909F908F9008958F9207
:102170009F92AF92BF92CF92DF92EF920F931F93F5
:102180001F921F921F930F934A015A01D12CC12C09
:1021900032E0E32E022F26E040E80E94EF0E0F907F
:1021A0000F900F900F901F910F91EF90DF90CF90B5
:1021B000BF90AF909F908F9008958F929F92AF9213
:1021C000BF92CF92DF92EF920F93C42ED12C1F9229
:1021D0001F921F921F92912C812CB12CA12CE12CCB
:1021E000062F21E043E2FC016285828193810E94F7
:1021F000EF0E0F900F900F900F900F91EF90DF90D8
:10220000CF90BF90AF909F908F9008958F929F92A4
:10221000AF92BF92CF92DF92EF920F93C62ED12C46
:102220001F921F925F934F9324E0822E912C34E0F3
:10223000A32EB12CE12C00E020E043EAFC016285F2
:10224000828193810E94EF0E0F900F900F900F905C
:102250000F91EF90DF90CF90BF90AF909F908F90B5
:1022600008958F929F92AF92BF92CF92DF92EF929A
:102270000F93C42ED12C1F921F921F921F92912C4C
:10228000812CB12CA12CE12C062F23E043E2FC0190
:102290006285828193810E94EF0E0F900F900F90C4
:1022A0000F900F91EF90DF90CF90BF90AF909F90E5
:1022B0008F900895CF92DF92FF920F931F93CF9349
:1022C000DF9300D000D0CDB7DEB78C01F62E198297
:1022D0001A821B821C82462F61E10E94DD104F2D65
:1022E00060E1C8010E94DD104F2D64E0C8010E942A
:1022F000311183E0C82ED12CAE014F5F5F4F6F2D9F
:10230000C8010E940611811114C089819A81AB8194
:10231000BC819D7F83309140A041B10551F064E6BE
:1023200070E080E090E00E94740981E0C81AD10852
:1023300019F74F2D64E1C8010E94DD104F2D60E1B7
:10234000C8010E94DD1064E170E080E090E00E942E
:1023500074090F900F900F900F90DF91CF911F9104
:102360000F91FF90DF90CF9008952F923F924F9260
:102370005F926F927F928F929F92AF92BF92CF9215
:10238000DF92EF92FF920F931F93CF93DF93CDB71E
:10239000DEB7E8970FB6F894DEBF0FBECDBFDC0105
:1023A0001A963C91311125C1922E242E362E3C01D5
:1023B000FC01E280F380D701ED91FC910190F08166
:1023C000E02D60E0C70109958C01009709F414C164
:1023D000FC01C080D180C114D10409F410C15301A3
:1023E000F4E0AF0EB11CDC011196BC92AE921496D3
:1023F0009C92FE0131962F019F0148E050E060E081
:10240000D30112968D919C910E949310982EF80101
:1024100014828111FAC08D8191ED992E893059F580
:102420008980D701ED91FC910280F381E02D222D6E
:1024300041E0632DC7010995F3018287882309F4E0
:10244000E1C098859583682F828193810E946310F3
:10245000982ED801CD92DC92882339F1D701ED91E5
:10246000FC910480F581E02DD3011A966C91C7018F
:102470000995F3011286892DE8960FB6F894DEBF10
:102480000FBECDBFDF91CF911F910F91FF90EF90C5
:10249000DF90CF90BF90AF909F908F907F906F9084
:1024A0005F904F903F902F900895811082C09501CA
:1024B00042E0F3016285828193810E943708982E61
:1024C0008111D9CF1F921F925F924F9258E0852EB3
:1024D000912C68E0A62EB12CD12CC12C79E2E72EEC
:1024E00000E026E040EAF3016285828193810E9448
:1024F000EF0E982E0F900F900F900F908111BBCF81
:102500008B81D3011B968C931B97820120E048E0BE
:1025100050E01A966C911A9712968D919C910E9498
:10252000B710982E8111A7CF4B815C8120E0F30179
:102530006285828193810E94B710982E81119BCF72
:10254000498150E08E010F5D1F4F20E0D3011A96A4
:102550006C911A9712968D919C910E94B710982EAB
:10256000811189CF1F921F921F921F92912C812C53
:10257000B12CA12CE12C0E8129E040E0F301628511
:10258000828193810E94EF0E982E0F900F900F90F2
:102590000F90811170CF11E0D3011B968C911B9786
:1025A0008117D0F0412F68E0C3010E9431111F5FF5
:1025B000F3CF482D413208F040E250E09201D301C0
:1025C0001A966C911A9712968D919C910E94931075
:1025D000982E811150CF6BCF1296ED91FC911397ED
:1025E000EA58FF4F80818460808381E050968C930D
:1025F00042CF49ED942E3FCF36ED932E3CCF27EDC1
:10260000922E39CF84ED982E36CFD182C08233CF2F
:102610002F923F924F925F926F927F928F929F92F2
:10262000AF92BF92CF92DF92EF92FF920F931F93E0
:10263000CF93DF93CDB7DEB7C358D1090FB6F89467
:10264000DEBF0FBECDBFDC0116963C913111FEC13D
:10265000022FA42EB62E3C01FC01C480D580118E21
:10266000D601ED91FC910190F081E02D60E0C60172
:1026700009952C010097E9F4E6EDFE2E8F2DCD573C
:10268000DF4F0FB6F894DEBF0FBECDBFDF91CF9105
:102690001F910F91FF90EF90DF90CF90BF90AF9080
:1026A0009F908F907F906F905F904F903F902F9072
:1026B0000895FC01E080F180E114F10409F4C9C13E
:1026C0001301F7E02F0E311CDC0111963C922E9283
:1026D00014960C939E0126593F4F48E050E060E06D
:1026E000F301848195810E949310182F8111B7C145
:1026F000AB961FADAB97D201ED92FC92D601ED9156
:10270000FC910280F381E02D2A2D40E06B2DC60163
:102710000995F3018683882309F49EC1E2969FAD53
:10272000E2979087682F848195810E946310F82E2C
:10273000D601ED91FC91D20114961C92882359F098
:102740000480F581E02DD30116966C91C6010995A0
:10275000F301168293CF0190F081E02DD3011696FC
:102760006C91C6010995009709F486CFFC0104839A
:10277000910141E0D30116966C91169714968D91B4
:102780009C910E9437081111A4C0EC96BFADEC9744
:10279000CF57DF4FB883C158D0402E01E1E44E0E31
:1027A000511CC3010296CE57DF4F99838883C258CC
:1027B000D040D2015096EE96BFAFAEAFEE97CF5756
:1027C000DF4FF881C158D040FF1509F49EC0E0E208
:1027D000F1E0D2011196FC93EE93CE57DF4F888142
:1027E0009981C258D04013969C938E931297149659
:1027F0001C92149719961C9219971A961C921A9764
:102800001D961C921D971F961C921E921E979096C5
:102810001C92909791961C92919792961C929297E7
:1028200098961C929897EE96EEADFFADEE971696A1
:10283000FC93EE9315971896FC93EE9317971C96BE
:10284000FC93EE931B97D30114960D90BC91A02D91
:10285000C258DF4FB983A883CE57D040F301F68129
:10286000C058DF4FF883C058D0408E010F5F1F4F14
:102870002F2D49E050E06F2FCD010E94B71081113C
:1028800021C0AB80BC805F924F921F930F9360E496
:10289000862E912CD12CC12C72E0E72E0F2D26E034
:1028A00040E8C058DF4F6881C058D040C258DF4F61
:1028B00088819981CE57D0400E94EF0E0F900F90E3
:1028C0000F900F90D30153968C918230F1F0F394D6
:1028D00076CF133108F012E1412F50E09E012659C6
:1028E0003F4FF3016681848195810E949310182FD8
:1028F000882309F44ACFD301ED91FC910480F5813E
:10290000E02DC3010995F12EB9CEF301838911EDB4
:10291000823089F7910142E06681848195810E942D
:10292000370868EE73E080E090E00E9474091F921F
:102930001F921F921F92912C812CB12CA12CD12C73
:10294000C12CE12CD30150960C91509729E040E026
:1029500016966C91169714968D919C910E94EF0E8D
:10296000182F0F900F900F900F908111C4CF68EE29
:1029700073E080E090E00E947409F301C784D12CD9
:102980001F921F921F921F92028D2BE041E26681DF
:10299000848195810E94EF0E0F900F900F900F9001
:1029A000882319F0853009F04FC0D3011F96CC90D1
:1029B0001F97D12C1F921F921F921F92912C812C36
:1029C000B12CA12CE12C00E02AE041E216966C919A
:1029D000169714968D919C910E94EF0E0F900F9078
:1029E0000F900F90882311F0853071F5FE01EF5B99
:1029F000FF4F86E291E091838083D3011F96CC90B4
:102A00001F97D12CFF93EF93CE0101969F938F9345
:102A100030E4832E912C40E8A42EB12C52E2E52E16
:102A200000E026E041E816966C91169714968D9179
:102A30009C910E94EF0E81E0F301808F0F900F9028
:102A40000F900F90F12C1ACE182F55CF29EDF22EA2
:102A500015CE97EDF92E12CE84EDF82E0FCEF201A1
:102A6000F182E08248CF8F929F92AF92BF92CF9235
:102A7000DF92EF920F93FC01C784D12C1F921F921B
:102A80007F936F9388248394912CAA24A394B12CD0
:102A900022E0E22E00E029E041E266818481958116
:102AA0000E94EF0E0F900F900F900F900F91EF90EC
:102AB000DF90CF90BF90AF909F908F900895CF936D
:102AC000DF931F92CDB7DEB78983809155058823A8
:102AD00039F0BE016F5F7F4F8DE395E00E943315A3
:102AE00080913A05882339F0BE016F5F7F4F82E203
:102AF00095E00E94331580911F05882339F0BE01AF
:102B00006F5F7F4F87E095E00E9433158091040549
:102B1000882339F0BE016F5F7F4F8CEE94E00E94F6
:102B200033150F90DF91CF9108952F923F924F92DE
:102B30005F926F927F928F929F92AF92BF92CF924D
:102B4000DF92EF92FF920F931F93CF93DF93CDB756
:102B5000DEB768970FB6F894DEBF0FBECDBF1B8AF5
:102B600038E03C8B3CE33D8B8A3F3FEF9307D9F441
:102B700016ED812F68960FB6F894DEBF0FBECDBF5D
:102B8000DF91CF911F910F91FF90EF90DF90CF9049
:102B9000BF90AF909F908F907F906F905F904F907D
:102BA0003F902F900895222E642E362E7C01DC015A
:102BB00016960D911C911797CE01439617969C93EC
:102BC0008E9316971A962C939E012F5F3F4F42E1EA
:102BD00050E060E0C7010E949310782EF701178340
:102BE0000683182F8111C5CF49845A848B849C8415
:102BF000FD81FF8B3E81388F670186E5C80ED11CB1
:102C000056011E8AD5018D919D915D010097D1F5E8
:102C1000BE89BF5FBE8BB031A9F7F601819191915A
:102C20006F01009709F06EC07394F0E17F12F5CF49
:102C3000F7018681978117ED892B09F49ACF2286B7
:102C4000262D40E0632DC7010E94CB07082F14ED0D
:102C5000882309F48ECF682FC7010E9420080097AF
:102C600009F486CFDC0114962C92602FC7010E94D4
:102C70006310182F882309F47CCF602FC7010E94AE
:102C8000A90777CFDC01ED91FC910084F185E02D5F
:102C900009958111BDCFF501929182918F01DC01DF
:102CA000ED91FC910088F189E02D688D09958823CC
:102CB00009F4AECFF80180819181DC01ED91FC91A6
:102CC0000484F585E02DA401B2010995882361F003
:102CD000022D262D432D6E89C7010E94DF0B182F70
:102CE000813D09F495CF45CFF80180819181DC01C8
:102CF000ED91FC910684F785E02D6F89099581118E
:102D0000E7CF86CFDC01ED91FC910084F185E02DC9
:102D10000995811189CFF601929182918F01DC0191
:102D2000ED91FC910088F189E02D688D0995811164
:102D30000DC0022D262D432D672DC7010E94DF0BEC
:102D4000182F877F813D09F014CF6ECFF801808165
:102D50009181DC01ED91FC910484F585E02DA401C5
:102D6000B2010995811160CFF80180819181DC0168
:102D7000ED91FC910684F785E02D6F8909958823F4
:102D8000C1F252CFCF92DF92EF92FF921F93CF9377
:102D9000DF93EC01162F7A01FA0180819181A281E3
:102DA000B3818130F3E09F07F1E0AF07B105C9F1CE
:102DB00070F48115E1E09E07AE07B10509F450C03B
:102DC00081309140A140B10561F180E041C0833084
:102DD00021E0920720E1A207B10529F0833093405A
:102DE000A041B10591F7412F64E1CE010E94DD10B1
:102DF000412F60E1CE010E94DD1064E170E080E0CF
:102E000090E00E9474096A85F7012181269521705E
:102E10006770412F8A819B810E9495151092B302A1
:102E2000D4CF8091B3028111D0CF412F61E1CE0187
:102E30000E94DD10412F60E1CE010E94DD10412F84
:102E400064E0CE010E94311181E08093B30281EBF6
:102E5000DF91CF911F91FF90EF90DF90CF90089579
:102E6000462F61E1CE010E94DD10412F60E1CE01CD
:102E70000E94DD101092B3028A8587701770880F48
:102E8000880F880F182B09F4A0CFEA80FB80670118
:102E9000F6E5CF0ED11CD0E0C0E0D6018D919D911A
:102EA0006D010097C1F0DC01ED91FC910084F1858A
:102EB000E02D099518130FC0AB96CC0FDD1FCE0D7A
:102EC000DF1D88819981DC01ED91FC910480F58101
:102ED000E02D09957ACF2196C031D105F1F675CF55
:102EE000CF92DF92EF92FF920F931F93CF93DF93D6
:102EF000CDB7DEB72E970FB6F894DEBF0FBECDBFAD
:102F0000FC012089211111C010E0812F2E960FB6EF
:102F1000F894DEBF0FBECDBFDF91CF911F910F910F
:102F2000FF90EF90DF90CF9008957C010E945508AC
:102F3000F7010485158526853785601B710B820B8B
:102F4000930B97FDE1CF81E090E09E878D878E0106
:102F50000F5F1F4F9E01235F3F4F41E062858281DB
:102F600093810E94B80E182F811121C082E0D82EC3
:102F700001E089818D2139F119861A861B861C860C
:102F8000AE01475F5F4F602FC7010E940611C82E38
:102F9000811119C0AE01475F5F4F602FC7010E94CA
:102FA000C216813B19F0882371F0C82E1C2D0E9497
:102FB00055086C597F4F8F4F9F4FF7016487758776
:102FC00086879787A2CFDD0C0F5F083091F601E06E
:102FD000F7018385801758F319861A861B861C868D
:102FE000AE01475F5F4F602FC7010E940611D82EC8
:102FF000811117C089859A858770917081309140C1
:1030000081F48B859C8581609C878B87AE01475FAF
:103010005F4F602FC7010E94C216813B29F08111CA
:1030200002C00F5FD5CFD82E1D2DC1CFCF93809179
:103030003E0483FF7EC083E094E00E94750280918D
:1030400043041F928F938EEF93E09F938F930E9480
:103050000E038CEF93E00E94750280914404282FA8
:10306000082E000C330B3F938F9389EF93E09F93CF
:103070008F930E940E0387EF93E00E947502809168
:103080004504282F082E000C330B3F938F9384EFB9
:1030900093E09F938F930E940E0382EF93E00E9430
:1030A000750280914604282F082E000C330B3F93A5
:1030B0008F938FEE93E09F938F930E940E038DEE7C
:1030C00093E00E94750280914704282F082E000C7F
:1030D000330B3F938F938AEE93E09F938F930E94DD
:1030E0000E0387EE93E00E94750280913D041F92CB
:1030F0008F9384EE93E09F938F930E940E0382EE52
:1031000093E00E94750280913C041F928F938FED93
:1031100093E09F938F930E940E038CED93E00E94A7
:1031200075028DB79EB74C960FB6F8949EBF0FBE32
:103130008DBFE0913F04F0914004309751F0C09171
:1031400043040480F581E02D83E494E00995C09365
:1031500043040E9474089093420480934104CF91E9
:1031600008951092360410923504E6E9F2E01182D7
:103170001282138214821582168217820E94D8034B
:1031800085E0E3E4F4E0DF011D928A95E9F710920F
:103190003D0410923C040E94161890E080E00E94CA
:1031A0006E0590E080E00C9458050F931F93CF9329
:1031B000DF93CDB7DEB7AA970FB6F894DEBF0FBE88
:1031C000CDBF8091EF02882309F452C11091E9002C
:1031D0001F708091EC0080FF39C080E8182B10929E
:1031E000E9008091E80083FF40C1E7EEF2E08FEE56
:1031F00092E02091F10021938E179F07D1F78091E3
:10320000E802833009F470C018F5813009F447C032
:10321000823009F4DEC08091E80083FF18C18091FC
:10322000E7029091E8029A3008F011C1E92FF0E02E
:10323000E45EF64E0C94692DFA19201A271A201A0A
:10324000271A821AA41A271AA31BB01B80E0C6CF24
:103250008A3009F4ADC08B3009F47DC08930D9F6CD
:103260008091E7028132B9F68091EB029091EC02F5
:10327000892B89F68091E800877F8093E800809110
:10328000E80082FF2CC08091F1008093DB028091E6
:10329000E8008B778093E8000E943D06BCCF8091C8
:1032A000E702813A09F0B7CF8091E800877F8093E9
:1032B000E8008091EB029091EC02892B61F060E0D4
:1032C00090E080E070E00E94AF058091E8008B778D
:1032D0008093E800A0CF68E08CED92E0F3CF80917E
:1032E000EF028111CCCF97CF8091E702813A09F0AC
:1032F00092CF8091EB029091EC02892BA1F4809106
:10330000E800877F8093E8008091E80080FFFCCF91
:10331000809111018093F1008091E8008E77809375
:10332000E8000E943D068091EB029091EC0201972B
:1033300009F071CF8091E800877F8093E800809149
:10334000E80080FFFCCF809110018093F100809114
:10335000E8008E779FCF8091E702813209F05BCF42
:103360008091EB029091EC02892B69F48091E80046
:10337000877F8093E8000E943D068091E902809358
:1033800011010E94B1188091EB029091EC0201971B
:1033900009F041CF8091E800877F8093E8000E9488
:1033A0003D068091E902809310010E94B11833CF4D
:1033B0008091E702813209F02ECF8091E800877F6B
:1033C0008093E8000E943D068091EA028093DA0231
:1033D00022CF8091E702813A09F01DCF8091E80069
:1033E000877F8093E8008091E80080FFFCCF809188
:1033F000DA02ABCF803889F0823849F58091EB0250
:103400008F70873020F58093E9008091EB0085FB79
:10341000882780F91092E90006C08091E40290911B
:10342000E502911182609091E800977F9093E80007
:103430008093F1001092F1008091E8008E7731C006
:10344000282F2D7F21F48823F1F0823079F18091AB
:10345000E80083FF0AC08091E800877F8093E8003E
:103460008091EB0080628093EB001F701093E90065
:10347000AA960FB6F894DEBF0FBECDBFDF91CF91F5
:103480001F910F9108958091E902813001F79330E7
:1034900009F080E08093E5021092E9008091E80055
:1034A000877F8093E8000E943D06D1CF8091E9029A
:1034B0008111F2CF8091EB028F702FEF280F263011
:1034C00030F68093E9002091EB0020FFE5CF9330A8
:1034D00031F48091EB0080628093EB00DDCF90911E
:1034E000EB0090619093EB0021E030E001C0220FEF
:1034F0008A95EAF72093EA001092EA008091EB00A7
:103500008860EACF8111A3CF0091E9020F77809103
:10351000E3008078802B8093E3008091E800877F30
:103520008093E8000E943D068091E80080FFFCCF78
:103530008091E30080688093E30083E0011101C083
:1035400082E08093EF0283CF8058823008F07FCFF3
:103550002091E9023091EA022C3D83E03807A1F581
:1035600083E08A838AE289834FB7F894DE01139659
:1035700020E03EE051E2E32FF0E050935700E49169
:1035800020FF03C0E295EF703F5FEF708E2F90E059
:10359000EA30C0F0C7968D939D932F5F243159F781
:1035A0004FBF8091E800877F8093E8006AE270E077
:1035B000CE0101960E94AF058091E8008B77809341
:1035C000E80045CFC096E7CF8091EB029091EC02E6
:1035D000432F55274330510509F44FC078F541304A
:1035E000510509F445C084E590E0EAE2F2E042309A
:1035F000510509F02CCF2091E800277F2093E800A7
:103600002091ED023091EE028217930708F49C019D
:1036100040E02115310509F063C0411161C080917E
:10362000E80082FDC9CF8091EF02882329F285301E
:1036300019F28091E80083FFF2CFBECF41325105ED
:1036400009F43FC04232510509F001CF83309105A2
:1036500008F0FDCEFC01EE0FFF1FE55DFE4F01906F
:10366000F081E02D885D9E4FDC018C9190E01DC0C3
:1036700082E190E0EEE7F2E0BECF33272130310562
:10368000C1F060F02230310509F0E1CEE0E9F2E06E
:10369000E4918E2F90E0E0E9F2E007C0E8EDF2E07F
:1036A000E4918E2F90E0E8EDF2E0009709F4CFCEA0
:1036B000A2CFEEECF2E0E4918E2F90E0EEECF2E09F
:1036C000F4CF8330910508F0C2CE880F991FFC011A
:1036D000EF5CFE4F0190F081E02D89E090E08BCF10
:1036E0008091EF02882309F467CF853009F464CF15
:1036F0008091E80083FD60CF8091E80082FD8FCF4C
:103700008091E80080FF85CF8091F3009091F200D6
:103710008927982789272115310519F088309105C7
:1037200050F041E0089709F040E08091E8008E7782
:103730008093E8006ECF44914093F1003196215080
:1037400031090196E8CF803809F081CE8091E800F8
:10375000877F8093E8008091E6028093F1006CCE31
:10376000811175CE0091E902023008F070CE80918F
:10377000E800877F8093E8000093E6020E943D0600
:10378000002399F084E08093EF0242E061EC81E055
:103790000E945C0642E061EC82E00E945C0646E228
:1037A00061EC83E00E945C0652CE8091E30087FDCD
:1037B000E9CF81E0E8CFEF92FF920F931F93CF9371
:1037C0007C018B010E940E06C82F811119C08091C7
:1037D000E80085FD0DC08091E8008E778093E800B9
:1037E0000E94D5180E940E06882389F3C82F08C0AE
:1037F000F70181917F018093F1000150110939F7A0
:103800008C2FCF911F910F91FF90EF900895AF9261
:10381000BF92CF92DF92EF92FF920F931F93CF93BD
:103820006091EA047091EB044091DE045091DF0452
:103830002091D2043091D3048091C6049091C704A2
:10384000E091A902F091AA026E177F07B1F4E0910E
:10385000A702F091A802E417F50779F4E091A50218
:10386000F091A602E217F30741F4E091A302F09170
:10387000A402E817F90709F45FC07093AA026093E5
:10388000A9025093A8024093A7023093A602209366
:10389000A5029093A4028093A30288E0EBEAF2E0F1
:1038A000DF011D928A95E9F72091E2043091E3044B
:1038B0004091E4045091E5046091E6047091E704BE
:1038C0008091E8049091E9040E94DF0D2091D604D4
:1038D0003091D7044091D8045091D9046091DA0412
:1038E0007091DB048091DC049091DD040E94DF0D77
:1038F0002091CA043091CB044091CC045091CD0466
:103900006091CE047091CF048091D0049091D10445
:103910000E94DF0D2091BE043091BF044091C0048D
:103920005091C1046091C2047091C3048091C40499
:103930009091C5040E94DF0D0E9474087C010E94D2
:10394000560D80914804813009F45EC008F460C0CF
:10395000823029F0833009F463C0C0E017C0C0E0B2
:1039600080919904807F803189F40E9455086853C2
:103970007F4F8F4F9F4F60939E0270939F02809363
:10398000A0029093A10280E2809399048EEAC82E4F
:1039900085E0D82E9EECA92E95E0B92E8601F8017F
:1039A000819191918F01009739F0DC01ED91FC91AB
:1039B0000680F781E02D0995A016B10681F7809168
:1039C0009904803409F4B8C068F5803209F49EC0C7
:1039D000803309F4ABC0813109F042C01092CE05AA
:1039E000F601819191916F01009739F0DC01ED9121
:1039F000FC910480F581E02D0995C016D10681F770
:103A000082E1809399042CC083E180939904A5CF2F
:103A100080919904807F803109F49FCF81E1F5CFB7
:103A2000C1E09ECF813509F49AC0803809F4AAC05C
:103A30008035B1F488EC0E947D0C86FF11C081E5D1
:103A4000809399040E9455086C507E4F8F4F9F4F72
:103A500060939E0270939F028093A0029093A102B4
:103A60002FB7F8948091370490913804A0913904CD
:103A7000B0913A042FBF8E199F098536910560F0E9
:103A80009F938F9389EA91E09F938F930E940E03F7
:103A90000F900F900F900F90809199049091A20237
:103AA000981749F18093A2021F928F9388E991E0C1
:103AB0009F938F930E940E030F900F900F900F9083
:103AC0008091A2028039B9F480914804823009F0D3
:103AD00069C083E191E09F938F938DE891E09F937C
:103AE0008F930E940E030E9484050E945F150F9021
:103AF0000F900F900F9081E0CF911F910F91FF9049
:103B0000EF90DF90CF90BF90AF9008950E9455083E
:103B100000919E0210919F022091A0023091A1027B
:103B2000601B710B820B930B97FD9ACF61E088EEBF
:103B30000E94CC0B80E465CF88EE0E947D0C80FD56
:103B40008FCF60E488EC0E94CC0B88ED0E947D0C46
:103B5000682F686088ED0E94CC0B80E552CF0E94F0
:103B6000550800919E0210919F022091A002309171
:103B7000A102601B710B820B930B97FD71CF80E844
:103B8000809399042C2F40E060E088E595E00E9446
:103B90009515882329F0823D09F462CF80EA31CF60
:103BA00080E92FCF88E191E096CFCF93DF938823F0
:103BB00009F454C09EE7980F933020F5C2E0D9E392
:103BC000823831F0C4E0D7E4833811F4C1E0D3E5A2
:103BD0000E9484058C2309F441C08D2F0E94BF03ED
:103BE0000E94D8032FEF41EE54E021504040504056
:103BF000E1F700C000008D2F0E94B303DF91CF9149
:103C00000C94D8039CEF980F913AB0F390E2980F80
:103C1000983088F4877021E030E0A90102C0440F99
:103C2000551F8A95E2F7CA01809590913604892341
:103C300080933604E3CF9BE5980F933030F490E007
:103C400080E0DF91CF910C946E05885A873130F473
:103C500090E080E0DF91CF910C945805DF91CF91F7
:103C60000895CF93DF93882309F4E9C09EE7980F66
:103C7000933020F5C2E0D9E3823831F0C4E0D7E4D4
:103C8000833811F4C1E0D3E50E9484058C2309F048
:103C9000D6C08D2F0E94BF030E94D8032FEF81EE64
:103CA00094E0215080409040E1F700C000008D2F4B
:103CB0000E94B303DF91CF910C94D8039CEF980F2F
:103CC000913A18F40E94BF03F5CF90E2980F983014
:103CD00068F4877021E030E001C0220F8A95EAF78E
:103CE00080913604822B80933604E4CF9BE5980FB5
:103CF000933080F4853A41F0863A49F083E890E0C9
:103D0000DF91CF910C946E0581E890E0F9CF82E8C5
:103D100090E0F6CF98E5980F973108F090C0883A78
:103D200009F448C0893A09F448C08A3A09F448C0FD
:103D30008B3A09F448C08C3A09F448C08D3A09F42A
:103D400048C08E3A09F448C08F3A09F448C0813B14
:103D500009F448C0803B09F448C0823B09F448C0DC
:103D6000833B09F448C0843B09F448C0853B09F40F
:103D700048C0863B09F448C0873B09F448C0883BEB
:103D800009F448C0893B09F448C08A3B09F448C09B
:103D90008B3B09F448C08C3B09F448C08D3B09F4C7
:103DA00048C08E3B09F448C090E080E0DF91CF919D
:103DB0000C94580582EE90E0F9CF89EE90E0F6CFB2
:103DC0008AEE90E0F3CF85EB90E0F0CF86EB90E0C9
:103DD000EDCF83EB90E0EACF84EB90E0E7CF87EB89
:103DE00090E0E4CF8CEC90E0E1CF8DEC90E0DECF82
:103DF00083E891E0DBCF8AE891E0D8CF82E991E0D7
:103E0000D5CF84E991E0D2CF81E292E0CFCF83E2B7
:103E100092E0CCCF84E292E0C9CF85E292E0C6CFB7
:103E200086E292E0C3CF87E292E0C0CF8AE292E0DE
:103E3000BDCF8FE690E0BACF80E790E0B7CFDF91BB
:103E4000CF910895CF92DF92EF92FF920F931F933D
:103E5000CF93DF9300D000D01F92CDB7DEB76C01B7
:103E600085E0F601DE01119601900D928A95E1F749
:103E7000F601408151812381348191E02115310582
:103E800031F05F3F19F491E04F3F09F090E090FD71
:103E900099C0F6010281F580F2949FE0F9224983EE
:103EA0005A830B83722F3D832C83602F8D810E9458
:103EB0000004182FE92FE295EF70EF3008F082C070
:103EC000F0E0EB59F04E0C94692D741F741FB21F73
:103ED000B21F28205A20E21FE21F4C21E21F22229B
:103EE0002222E21FE21FDE22F92FFF70FF2E907FB9
:103EF00019F0F29480EFF8220023C9F0FF2039F086
:103F000080913504F82AF09235040E94D803812F5D
:103F10000F900F900F900F900F90DF91CF911F9106
:103F20000F91FF90EF90DF90CF900C94311E812F76
:103F30000E94D51DFF2009F445C0F09480913504FE
:103F4000F822F09235040F900F900F900F900F9081
:103F5000DF91CF911F910F91FF90EF90DF90CF9065
:103F60000C94D803892F8F70907F903211F0829536
:103F7000807F112379F0113009F449C0002309F43E
:103F800055C0FF2059F0F601958190FF69C29F70DE
:103F9000958304C0002321F1F1100FC00F900F9002
:103FA0000F900F900F90DF91CF911F910F91FF9085
:103FB000EF90DF90CF900C944E0521E0F212EECFFF
:103FC000809334040F900F900F900F900F90DF911B
:103FD000CF911F910F91FF90EF90DF90CF900895B8
:103FE000F11011C0109234040F900F900F900F90A9
:103FF0000F90DF91CF911F910F91FF90EF90DF9085
:10400000CF900C94430591E0F912ECCFDBCF002365
:1040100049F0E5E0EF15B0F290913604982309F4E9
:10402000BDCFE2CFF4E0FF1568F2DECFFF20E1F272
:10403000812F0F900F900F900F900F90DF91CF91E5
:104040001F910F91FF90EF90DF90CF900C94D51DB2
:10405000892F869586958370C1F0813009F0B2CFA3
:10406000812F9370011102C090E080E00F900F90BB
:104070000F900F900F90DF91CF911F910F91FF90B4
:10408000EF90DF90CF900C945805812F9370011121
:1040900002C090E080E00F900F900F900F900F9073
:1040A000DF91CF911F910F91FF90EF90DF90CF9014
:1040B0000C946E05002309F471C0803FA1F40E94A6
:1040C00070038195809345040F900F900F900F908F
:1040D0000F90DF91CF911F910F91FF90EF90DF90A4
:1040E000CF900C941618813F19F40E947003EACF08
:1040F000823F31F40E947003819580934404E4CFA1
:10410000833F19F40E947003F8CF893F29F40E947D
:104110004E0380934604D8CF8A3F21F40E944E0379
:104120008195F7CF8B3F31F40E944E0381958093A8
:104130004704CACF8C3F19F40E944E03F8CF8091F8
:1041400043048160143FA1F0809143048260153FD5
:1041500079F0809143048460163F51F080914304CC
:104160008860173F29F0183F31F480914304806143
:1041700080934304A9CF80913C0481601D3F59F096
:1041800080913C0482601E3F31F01F3F09F09CCFBC
:1041900080913C04846080933C0496CF803FC1F4BE
:1041A0008091450487FD109245048091440481115B
:1041B0008BCF80914504811187CF80914604811176
:1041C00083CF8091470481117FCF10923D047CCF33
:1041D000813F29F48091450418162CF3E6CF809195
:1041E0004404123F29F487FFE0CF10924404DDCF4E
:1041F000133F19F41816CCF3D8CF193F39F4809136
:104200004604181694F610924604CFCF1A3F29F4AC
:104210008091460487FFC9CFF6CF1B3F39F48091C8
:10422000470487FFC2CF10924704BFCF1C3F29F439
:10423000809147041816BCF3B8CF809143048E7F59
:10424000143FA1F0809143048D7F153F79F0809158
:1042500043048B7F163F51F080914304877F173FC3
:1042600029F0183F31F4809143048F7E80934304FA
:104270009CCF80913C048E7F1D3F59F080913C047F
:104280008D7F1E3F31F01F3F09F08FCF80913C049E
:104290008B7F80933C0489CF892F837009F064C0A1
:1042A000011190CE812F829586958770880F880F97
:1042B000412F4F70C42ED12CF12CE12C082E04C0BC
:1042C000CC0CDD1CEE1CFF1C0A94D2F740E050E041
:1042D000BA0114FF11C00FE010E020E030E004C08C
:1042E000000F111F221F331F8A95D2F7B901A801B1
:1042F000409550956095709500912C0310912D0379
:1043000020912E0330912F039695969593709230BD
:10431000E9F028F5913089F04C295D296E297F2933
:10432000402351236223732340932C0350932D0386
:1043300060932E0370932F0345CEC02AD12AE22A20
:10434000F32A4C295D296E297F29EECF4C295D295E
:104350006E297F294027512762277327E5CF402305
:10436000512362237323EDCF8695002311F0892F0B
:104370008170882309F426CE812F829586958770D7
:10438000880F880F412F4F70C42ED12CF12CE12CB7
:10439000082E04C0CC0CDD1CEE1CFF1C0A94D2F7C6
:1043A00040E050E0BA0114FF11C00FE010E020E03F
:1043B00030E004C0000F111F221F331F8A95D2F76F
:1043C000B901A80140955095609570950091300312
:1043D00010913103209132033091330396959695D5
:1043E00093709230E9F028F5913089F04C295D29DD
:1043F0006E297F2940235123622373234093300386
:10440000509331036093320370933303DBCD0C2957
:104410001D292E293F29402B512B622B732BEECFC8
:104420004C295D296E297F29402751276227732750
:10443000E5CF40235123622373234C295D296E2944
:104440007F29DCCF803F09F44EC0D0F480E4810F97
:10445000803270F1002309F4ACC0FF2009F4A6C03B
:10446000812F0E94311E193309F099C0FFEF21EE10
:1044700084E0F15020408040E1F700C00000A2CD70
:10448000823F09F470C008F45BC0833F19F7002332
:1044900009F47CC0292F2F7181E090E0A0E0B0E00A
:1044A00004C0880F991FAA1FBB1F2A95D2F73AC0D4
:1044B000E12FE071FE2E892F8F71002351F00E94B1
:1044C000CD04812F8295807FF11068CD812F8F7070
:1044D00065CD0E94A904812F8295807FF11084CD43
:1044E000812F8F7081CD002331F1F4E0FF1508F4A6
:1044F00069CD292F2F7181E090E0A0E0B0E004C0E9
:10450000880F991FAA1FBB1F2A95D2F7409130032D
:1045100050913103609132037091330384279527C2
:10452000A627B7278093300390933103A0933203DB
:10453000B093330347CD25E02F1508F443CDD9CFF1
:10454000892F8F71002399F00F900F900F900F908B
:104550000F90DF91CF911F910F91FF90EF90DF901F
:10456000CF900C94CD04892F8F71002369F30F90A5
:104570000F900F900F900F90DF91CF911F910F919F
:10458000FF90EF90DF90CF900C94A904109230032D
:1045900010923103109232031092330313CD13356E
:1045A00009F464CF173409F00DCD60CF892F8F71D6
:1045B000CBCFF1103DCD892F8F71D9CF811102CD95
:1045C000002309F4FFCC0E94B1188FEF90E7E2E0DE
:1045D00081509040E040E1F700C000000E9490054B
:1045E000F89487E797E7909301088093000887E0A5
:1045F00090EBDC018093CF059093D005A093D1057B
:10460000B093D20588E19CE00FB6F894A89580930A
:1046100060000FBE90936000FFCF0F931F93CF9366
:10462000DF938091F902807FB9F48091F6028823AC
:1046300099F080912B031091FA026091F40270912D
:10464000F502C091F702D091F80221E06F3F09F026
:1046500020E006E0181305C0DF91CF911F910F9164
:10466000089531E0209721F0322F7F3F09F030E0AC
:1046700090E030FD33C0089FF001099FF00D112438
:10468000DF01A550BD4F11963C911197371326C0FD
:104690003C91361323C012963C91129731111EC0E3
:1046A00013964D915C914C1B5D0B483C5105B0F449
:1046B0008091F9028F7080618093F902E050FD4F84
:1046C00080818F708061808384EF92E00E94221F3E
:1046D000DF91CF911F910F910C94ED04019687709B
:1046E000B9CF9F92AF92BF92CF92DF92EF92FF929B
:1046F0000F931F93CF93DF93CDB7DEB761970FB6BC
:10470000F894DEBF0FBECDBF8C0185E0F801DE015D
:104710001D9601900D928A95E1F7F8014081518133
:10472000F280C380D4809091F4026091F5022091D0
:10473000F7023091F80281E02115310531F06F3F29
:1047400019F481E09F3F09F080E0F82FF1709F2E6F
:1047500080FD49C184EFA82E82E0B82EE090F602D9
:10476000F601E21BF30BEE2009F400C18091F9027F
:10477000782F707FE83CF10508F0BAC0711181C054
:10478000EF2C651322C0941320C0F1101EC08F704F
:1047900080618093F902C5010E94221F8091F90275
:1047A000F80185838E2D61960FB6F894DEBF0FBE9B
:1047B000CDBFDF91CF911F910F91FF90EF90DF90D0
:1047C000CF90BF90AF909F90089581E0C114D10425
:1047D00031F05F3F19F481E04F3F09F080E080FD48
:1047E00024C081E08F25F82FF170BF2E80FF3FC0DD
:1047F00080912B032091FA0236E0821318C07C2DA1
:10480000D98AC88A6F2D89890E940004292F229590
:104810002F70223000F1243028F59F7001F1F8014B
:104820009581907FE1F4E92CBDCF80E0DCCF90E072
:10483000389FF001399FF00D1124E550FD4F618143
:10484000561306C06081461303C062816F110FC00A
:1048500001968770D2CF9F7011F0882321F3805E7C
:10486000883008F3C8010E94221F9B2CDCCFFF2058
:1048700009F498CF8091F90281608093F902E12CCC
:1048800091CF651306C0941304C0F801FF2009F40A
:1048900088C04D875E87FF867C2DD98AC88A6F2D98
:1048A00089890E94F704882309F4ABC0FF2009F42A
:1048B000A8C08091F902803270F02091F40230910A
:1048C000F50238872F831986DB86CA868C87CE014E
:1048D00007960E94221F86E0F801A4EFB2E0019043
:1048E0000D928A95E1F70E940D23EE24E3945ACFAE
:1048F00071110AC084EF92E00E94221F86E0F50148
:1049000011928A95E9F7BBCF65130FC094130DC0C0
:10491000F1100BC0F8018583C8010E94221F86E0B8
:10492000F50111928A95E9F73DCF4D875E87FF86A5
:104930007C2DD98AC88A6F2D89890E94F704882323
:1049400009F45FC0FF2009F45CC08091F902803255
:1049500010F22091F4023091F5023A8329831B82F0
:10496000DD82CC828E83CE010196B3CFE83CF10587
:10497000B0F6EF2CFF2009F444C065131FC0941358
:104980001DC08091F90280FD10C0982F907F69F0C2
:10499000F8018583903F31F0982F907F905F8F7062
:1049A000892B8583C8010E94221F86E0F801A4EFAD
:1049B000B2E001900D928A95E1F7F4CE4D875E87C3
:1049C000FF867C2DD98AC88A6F2D89890E94F704B9
:1049D000811181CF8091F90281608093F902C80131
:1049E0000E94221FDFCEFF2061F04D875E87FF8689
:1049F0007C2DD98AC88A6F2D89890E94F70481117C
:104A00006ACFC8010E94221F70CF1F93CF93DF93FC
:104A1000CDB7DEB767970FB6F894DEBF0FBECDBF38
:104A20004B8B5C8B6D8B7E8B8F8B1A8A198A85E002
:104A3000FE017396DE011D9601900D928A95E1F7B5
:104A400086E0FE013D96DE01179601900D928A9553
:104A5000E1F7CE0107960E947123811137C086E0ED
:104A6000FE013796DE01119601900D928A95E1F7CD
:104A70009F8188852A853B85232B39F08F3F19F448
:104A800081E09F3F19F080E001C081E080FD1EC001
:104A90002091FA0230E0C901019687709927409170
:104AA0002B034817190659F196E0929FD001939F66
:104AB000B00D1124A550BD4FFE01319601900D920D
:104AC0009A95E1F78093FA020E94ED0416E0809136
:104AD0002B039091FA028917F9F0819FC0011124EC
:104AE00085509D4F0E9471238823B1F080912B0344
:104AF00090E001968770992780932B03E8CF0E945E
:104B0000B1181092FA0210922B0386E0E4EFF2E063
:104B1000DF011D928A95E9F767960FB6F894DEBF1C
:104B20000FBECDBFDF91CF911F910895CF93DF933B
:104B300000D01F92CDB7DEB72091EF02243021F5CF
:104B400023E029839B838A8382E08093E9008FEFAF
:104B50009091E800815095FD06C095ED9A95F1F78A
:104B600000008111F5CF8091E80085FF0DC050E075
:104B700040E063E070E0CE0101960E94DB1B809173
:104B8000E8008E778093E8000F900F900F90DF91F0
:104B9000CF910895CF93DF9300D01F92CDB7DEB7AA
:104BA0002091EF02243061F519821A821B8222E0E3
:104BB00029838138910520F0805891099B838A834D
:104BC00082E08093E9008FEF9091E800815095FD9D
:104BD00006C095ED9A95F1F700008111F5CF80910F
:104BE000E80085FF0DC050E040E063E070E0CE01DA
:104BF00001960E94DB1B8091E8008E778093E8008D
:104C00000F900F900F90DF91CF9108952091EF02B8
:104C1000243049F522E02093E9002FEF3091E8009D
:104C2000215035FD06C035ED3A95F1F70000211110
:104C3000F5CF2091E80025FF16C02091100150E02B
:104C400040E063E070E0222339F021E02093F1009E
:104C500050E040E065E070E00E94DB1B8091E800DE
:104C60008E778093E8000895CF93DF932091EF0231
:104C7000243011F521E02093E90021E8215021F0B2
:104C80003091E80035FF1BC02091E80025FF14C0DB
:104C9000EC0150E040E068E070E00E94DB1B809196
:104CA000E8008E778093E80088E0FE01ACEDB2E08A
:104CB00001900D928A95E1F7DF91CF910895EFE38E
:104CC000F1E03197F1F700C00000D8CFAF92BF926A
:104CD000CF92DF92EF92FF920F931F93CF93DF93C8
:104CE0006C01CB01E22EDB01ED91FC910084F1859A
:104CF000E02D09951F928F938BED91E09F938F93F9
:104D00000E940E03E801E00EF12EF11C0F900F90AF
:104D10000F900F9085EDA82E81E0B82ECE15DF05FF
:104D200061F089911F928F93BF92AF920E940E0300
:104D30000F900F900F900F90F1CF82ED91E09F9325
:104D40008F930E940E030F900F90F80182818130A3
:104D500099F488EB91E09F938F930E940E030F903C
:104D60000F90DF91CF911F910F91FF90EF90DF9007
:104D7000CF90BF90AF900895D601129688E0019031
:104D80000D928A95E1F70E945508D6011B967C93F7
:104D90006E931A97E6CF6F927F928F929F92AF9207
:104DA000BF92CF92DF92EF92FF920F931F93CF9318
:104DB000DF9300D0CDB7DEB77C01CDB6DEB6DC0127
:104DC00058968C91811118C0912C892D0FB6F894AA
:104DD000DEBE0FBECDBE0F900F90DF91CF911F9121
:104DE0000F91FF90EF90DF90CF90BF90AF909F908A
:104DF0008F907F906F9008950E945508F7018488E6
:104E00009588A688B788681979098A099B0997FD4A
:104E1000DBCFADB6BEB64285838590E08134910587
:104E200008F045C09A83898389819A812DB73EB75E
:104E3000281B390B0FB6F8943EBF0FBE2DBF8DB7A0
:104E40009EB701968C019E012F5F3F4FD7011696AA
:104E50006C91169714968D919C910E94B80E982E85
:104E6000811113C029813A812330310570F0F70197
:104E700085859685009749F0DC01ED91FC910190C4
:104E8000F081E02D40E0B70109950FB6F894BEBE61
:104E90000FBEADBE0E945508F701218D620F711D36
:104EA000811D911D648B758B868B978B8ECF80E4D3
:104EB00090E0B8CFCF9310924C0410924B0488EE40
:104EC00093E0A0E0B0E080934D0490934E04A09353
:104ED0004F04B09350048FE591E090934A0480937F
:104EE00049048FEF9FEF909356048093550487E811
:104EF00091E090935905809358051092600581E0E8
:104F000080936105109262058AE595E090935F05B4
:104F100080935E0510925A0588E080935B058CE3D0
:104F200080935C0510925D05E8E5F5E0C1E08AE557
:104F300095E01586C687178694878387359625E082
:104F4000E33AF207B1F71092CE0581E1809399041C
:104F50008DE395E00E94170382E295E00E9417031B
:104F600087E095E00E9417038CEE94E00E941703FF
:104F700081E991E09093E1048093E0049093D5045B
:104F80008093D4049093C9048093C8049093BD0483
:104F90008093BC0481E791E09093AC048093AB04D0
:104FA00088E595E09093AE048093AD041092BB0425
:104FB0001092AF0488E08093B0049CE39093B10416
:104FC000C093B2048093B30484E08093B40410923D
:104FD000B5041092B6041092B7041092B80410925F
:104FE000B9041092BA04AEEAB5E0FD0190E080E0A9
:104FF00021913191232B09F044C0880F991FFC01A6
:10500000E255FA4F8BEA94E09183808381E791E047
:1050100090939B0480939A0488E595E090939D0477
:1050200080939C041092AA0410929E0488E08093BE
:105030009F049CE39093A00491E09093A10480933B
:10504000A20484E08093A3041092A4041092A50407
:105050001092A6041092A7041092A8041092A9041A
:1050600090E080E02D913D91232B89F4880F991FCA
:10507000FC01E255FA4F8AE994E091838083CF9155
:10508000089501968031910509F0B2CFBFCF019606
:105090008031910539F7F3CF1F920F920FB60F921F
:1050A00011248F939F93AF93BF9380913B04811101
:1050B00013C08091370490913804A0913904B091C5
:1050C0003A044196A11DB11D809337049093380492
:1050D000A0933904B0933A04BF91AF919F918F91FF
:1050E0000F900FBE0F901F9018951F920F920FB642
:1050F0000F9211242F933F934F935F936F937F935E
:105100008F939F93AF93BF93EF93FF938091E100B1
:1051100082FF09C08091E20082FF05C08091E1001A
:105120008B7F8093E1008091DA0080FF1FC0809127
:10513000D80080FF1BC08091DA008E7F8093DA0058
:105140008091D90080FF9DC080E189BD82E189BD49
:1051500009B400FEFDCF81E08093EF028091D80278
:10516000811104C00E9490050E948E068091E1008A
:1051700080FF1FC08091E20080FF1BC08091E20091
:105180008E7F8093E2008091E20080618093E20054
:105190008091D80080628093D80019BC85E080930C
:1051A000EF028091DB028093D9021092DB020E9411
:1051B000B1188091E10084FF2DC08091E20084FF4E
:1051C00029C080E189BD82E189BD09B400FEFDCF1F
:1051D0008091D8008F7D8093D8008091E1008F7EF0
:1051E0008093E1008091E2008F7E8093E2008091C5
:1051F000E20081608093E2008091E602882309F456
:1052000046C084E08093EF020E94B1188091D902D9
:105210008093DB028091E10083FF22C08091E20055
:1052200083FF1EC08091E100877F8093E10082E0D0
:105230008093EF021092E6028091E1008E7F8093CE
:10524000E1008091E2008E7F8093E2008091E20095
:1052500080618093E20042E060E080E00E945C06B2
:10526000FF91EF91BF91AF919F918F917F916F913E
:105270005F914F913F912F910F900FBE0F901F9014
:10528000189519BC1092EF021092D8026FCF80913E
:10529000E30087FD02C081E0B5CF83E0B3CFCF93B9
:1052A000DF93CDB7DEB72A970FB6F894DEBF0FBEF7
:1052B000CDBF84B7877F84BF0FB6F894A89580913F
:1052C0006000886180936000109260000FBE80E8EB
:1052D00090E00FB6F89480936100909361000FBE48
:1052E00080E799E0909395018093940186E091E0A6
:1052F0009093400480933F0485E092E00E94750201
:105300000E9490050E948E06789482E084BD93E00E
:1053100095BD9AEF97BD80936E0080913E048160A9
:1053200080933E04269A0E94A60B219A229A2398E3
:10533000209A80E58CBD81E08DBD259868E188E8E4
:105340000E94CC0B60E288E70E94CC0B60E088E70B
:105350000E94CC0B10E000E088E60E947D0C0F5FFD
:105360001F4F80FF1CC061EC88ED0E94CC0B60E2F7
:1053700080ED0E94CC0B64E088EE0E94CC0B88EE9E
:105380000E947D0C82FFFBCF0E94560D60E288ECEC
:105390000E94CC0B61E080E80E94CC0B03C00F3F61
:1053A0001007D1F680EE94E090934B0580934A0568
:1053B00084ED94E09093300580932F0588EC94E081
:1053C00090931505809314058CEB94E09093FA0468
:1053D0008093F9048091EF02843009F0DBC00E94D1
:1053E0006108882309F4D6C083EF91E00E9475021A
:1053F00085EE91E00E94750277247A9423E0622E74
:1054000030E1532E48E1C42ED12C8091EF0285303B
:1054100009F4C3C00E94071C06EB12E0412C842D46
:105420000E94B10D4C01F801A080B1808A159B0546
:1054300071F1312CEE24E394F12CA824B924C50198
:105440008E219F21892BE9F03E824F8221E0C70106
:1054500088219921892B09F420E028870E9474086B
:105460008160782F9A8789874E815F8168858A85D8
:105470000E940525F801808191818E259F259183C9
:1054800080833394EE0CFF1CF0E13F12D8CF43949D
:105490000E5F1F4F40E14412C2CF79827A821B8295
:1054A0000E9474088160782F9D838C8349815A8182
:1054B0006B818D810E940525209141043091420429
:1054C0004FB7F8948091370490913804A091390433
:1054D000B0913A044FBFFC01E21BF30B9F01809196
:1054E0003D0442E350E0811102C04CE251E0241738
:1054F000350780F09091440410914504F0904604E3
:1055000000914704911183C0111146C1F11044C1AB
:10551000011142C10E9484059091B502891731F0B2
:105520000E9484058093B5020E945F152091E400DB
:105530003091E5008091D6029091D7022817390763
:1055400031F18091E4009091E5009093D70280932F
:10555000D6020E9461088823D1F08091EF02843046
:10556000B1F48091E9008F709091EC0090FFBDC084
:1055700090E8892B6092E9009091EB0090FF04C0C5
:105580009091EE0097FDCFC08F708093E9000E944C
:10559000D5183BCF0E94D5181DCF8091EF028430E3
:1055A00011F110923B0480E40FB6F894A895C092D4
:1055B00060000FBE8093600083B7817F846083BFEB
:1055C00083B7816083BF7894889583B78E7F83BFCC
:1055D0000FB6F894A8958091600088618093600070
:1055E000109260000FBE8091E502882369F00E944E
:1055F000071C10E0812F0E94B10D892B09F0B7C064
:105600001F5F1031B9F701CF0E94071CFECE8F3FFC
:1056100019F08F5F80933D04191624F40E947003E3
:10562000809344048091440487FF05C00E94700366
:10563000819580934404111624F40E947003809392
:1056400045048091450487FF05C00E947003819541
:105650008093450460914404662331F11091450420
:10566000112311F1062E000C770B880B990B0E9469
:10567000332C23E333E343E35FE30E94C02C0E9417
:10568000FB2B60934404612F110F770B880B990B50
:105690000E94332C23E333E343E35FE30E94C02CF7
:1056A0000E94FB2B609345041F1424F40E944E03B8
:1056B000809346048091460487FF05C00E944E03F4
:1056C000819580934604101624F40E944E03809323
:1056D00047048091470487FF05C00E944E038195CF
:1056E000809347040E94161815CF90E042CFE091B6
:1056F0000101F0910201E90FF11D20819F5F3091BE
:1057000005019323909304012093F1009091E80008
:1057100095FD09C09091E80090FF05C09091E800C8
:105720009E779093E800909104012091030129173E
:1057300021F02091E80025FDDACF2091F30090912F
:10574000F200322F292F232B09F41ECF9091E8006D
:1057500090FF1ACF9091E80095FD06C09091E80067
:105760009E779093E80010CF1092F100F3CF59BCD0
:1057700082E189BD09B400FEFDCF8091D8008F7D04
:105780008093D8008091E00082608093E000809157
:10579000E00081FDFCCF39CE8F3F09F03ACF4BCFEF
:1057A00078941F920F920FB60F9211248F939F93AC
:1057B000AF93BF938091370490913804A09139043E
:1057C000B0913A040196A11DB11D809337049093C6
:1057D0003804A0933904B0933A04BF91AF919F91DC
:1057E0008F910F900FBE0F901F9018950E946E2CF6
:1057F00008F481E008950E94022C6894B1110C9481
:10580000B52C08950E949A2C88F09F5798F0B92FD4
:105810009927B751B0F0E1F0660F771F881F991FE5
:105820001AF0BA95C9F714C0B13091F00E94B42CA7
:10583000B1E008950C94B42C672F782F8827B85FB7
:1058400039F0B93FCCF3869577956795B395D9F73D
:105850003EF490958095709561957F4F8F4F9F4F47
:105860000895E89409C097FB3EF490958095709553
:1058700061957F4F8F4F9F4F9923A9F0F92F96E99C
:10588000BB279395F695879577956795B795F11111
:10589000F8CFFAF4BB0F11F460FF1BC06F5F7F4FAE
:1058A0008F4F9F4F16C0882311F096E911C07723C0
:1058B00021F09EE8872F762F05C0662371F096E8C9
:1058C000862F70E060E02AF09A95660F771F881F98
:1058D000DAF7880F9695879597F90895990F00083C
:1058E000550FAA0BE0E8FEEF16161706E807F907B2
:1058F000C0F012161306E407F50798F0621B730B4D
:10590000840B950B39F40A2661F0232B242B252BCD
:1059100021F408950A2609F4A140A6958FEF811D70
:10592000811D089557FD9058440F551F59F05F3F52
:1059300071F04795880F97FB991F61F09F3F79F0B1
:1059400087950895121613061406551FF2CF469533
:10595000F1DF08C0161617061806991FF1CF8695B5
:105960007105610508940895E894BB276627772799
:10597000CB0197F908950E946E2C08F48FEF0895DB
:105980000E94D32C0C94442D0E94362D38F00E9496
:105990003D2D20F0952311F00C942D2D0C94332DDA
:1059A00011240C94B52C0E94922C70F3959FC1F396
:1059B000950F50E0551F629FF001729FBB27F00DBD
:1059C000B11D639FAA27F00DB11DAA1F649F662712
:1059D000B00DA11D661F829F2227B00DA11D621F61
:1059E000739FB00DA11D621F839FA00D611D221F1B
:1059F000749F3327A00D611D231F849F600D211DFF
:105A0000822F762F6A2F11249F5750409AF0F1F081
:105A100088234AF0EE0FFF1FBB1F661F771F881FEA
:105A200091505040A9F79E3F510580F00C942D2DC8
:105A30000C94B52C5F3FE4F3983ED4F386957795AC
:105A40006795B795F795E7959F5FC1F7FE2B880F90
:105A5000911D9695879597F9089597F99F6780E826
:105A600070E060E008959FEF80EC089500240A94B0
:105A70001616170618060906089500240A94121629
:105A80001306140605060895092E0394000C11F45C
:105A9000882352F0BB0F40F4BF2B11F460FF04C009
:105AA0006F5F7F4F8F4F9F4F089597FB072E16F420
:105AB000009407D077FD09D00E946F2D07FC05D018
:105AC0003EF4909581959F4F0895709561957F4F15
:105AD0000895EE0FFF1F0590F491E02D0994AA1B85
:105AE000BB1B51E107C0AA1FBB1FA617B70710F0C9
:105AF000A61BB70B881F991F5A95A9F780959095FB
:0A5B0000BC01CD010895F894FFCF19
:105B0A000596010000FFEF0634260626CA259625CB
:105B1A000101FF66756C6C006C6F77000000000075
:105B2A00ED0900000000300B407F224D01CE00AC91
:105B3A00003C0255026E020000000008131F0E8985
:105B4A000BCB26860B1E0E1C0E810B7C0B730BA730
:105B5A000DA40D310BFEFF0000690B00000000DDF3
:105B6A0009C309E409E309EA09E709E709000000AA
:105B7A0000B5111F0E2D07701754075A111C0E4F2E
:105B8A00075308000000002008CB07A907000000FF
:045B9A00006626007B
:106800008800EA44E944E244040005000600070069
:10681000080009000A000B000C000D000E000F001C
:1068200010001100120013001400150016001700CC
:10683000180019001A001B001C001D001E001F007C
:10684000200021002200230024002500260027002C
:10685000280029002A002B002C002D002E002F00DC
:10686000300031003200330034003500360037008C
:10687000380039003A003B003C003D003E003F003C
:1068800040004100420043004400450046004700EC
:10689000480049004A004B004C004D004E004F009C
:1068A000500051005200530054005500560057004C
:1068B000580059005A005B005C005D005E005F00FC
:1068C00060006100620063006400F1A18500670060
:1068D000680069006A006B006C006D006E006F005C
:1068E0007000710072007300890087008A008B00BD
:1068F000E000E100E200E300E400E500E600E7007C
:106900000100010001000100EA4401000100E2442D
:106910000100010001000100460001004A004B0097
:10692000010001004700480001000100E9440100A6
:106930000100010001000100010001003A003B00DC
:106940003C003D003E003F0040004100420043004B
:10695000010035004C0001000100440045005200D8
:1069600049000100010050004F0029004D004E0079
:1069700051000100010001000100010001000100BF
:1069800001000100010001000100010001000100FF
:1069900000E00100010001000100010001004D00C4
:1069A0004A004E004B0001000100010001000100FF
:1069B00001000100010001000100010001000100CF
:1069C00001000100010001000100010001000100BF
:1069D00001000100010001000100010001000100AF
:1069E0000100010001000100490001000100010057
:1069F000010001000100010001000100010001008F
:00000001FF
